:1000000054C019C4F9C124C46BC06AC069C068C0B7
:1000100067C066C065C064C063C062C03BC40403FF
:10002000090422037700770077002E007200650034
:10003000630075007200730069006F006E002E008F
:100040006A00700010035500530042002D0032007A
:10005000330032001201100102000008C016E10551
:10006000000101020001090243000201008032097F
:100070000400000102020100052400100104240212
:100080000205240600010524010301070583030876
:1000900000FF09040100020A000000070501020236
:1000A0000000070581020800000011241FBECFE5F3
:1000B000D2E0DEBFCDBF10E0A0E6B0E0EEEAFAE0AD
:1000C00002C005900D92AC36B107D9F711E0ACE64D
:1000D000B0E001C01D92AF33B107E1F758D3E5C4DA
:1000E0008FCFAC9A8BB780628BBF8BE480937C0000
:1000F0008093A7008AE580937B008093A6000895F3
:100100001F93CF93DF93DC01162FEA01888184FFD0
:1001100005C0898198E88927898302C08AE5888398
:10012000AE014E5F5F4F212FFA018D9181932150D7
:100130001216DCF3CA01612F48D11C5F1883DF91CE
:10014000CF911F91089546EA50E0DADF08954BE71A
:1001500050E0D6DF08951F93CF93DF9360918C001A
:10016000635067FDB3C080918900CCE0D0E0C81B2C
:10017000D109C057DF4F80918800803118F4CE013B
:10018000EAD29EC08D3209F08BC0683009F098C069
:1001900083EC809370008AE58093600010926C007D
:1001A0008881807621F0CE01A8D2282F66C09A815E
:1001B000109279008981882321F410927A0022E03C
:1001C00055C0853019F490938D004FC08630B9F535
:1001D0008B81813041F484E590E090938B00809393
:1001E0008A0022E128C0823021F4CE0171D2282F6A
:1001F00022C08330F9F48A81882341F48EE190E0B3
:1002000090938B0080938A0024E015C0813041F4E4
:1002100082E290E090938B0080938A0022E20BC0F0
:10022000823041F484E490E090938B0080938A00C4
:1002300020E101C020E080E480936C001EC0883083
:1002400021F421E08FE890E013C0893019F49093F5
:100250008F000BC08A3011F421E008C08B3029F4E4
:100260008BE480937C008093A70020E089E790E0F6
:1002700090938B0080938A0009C02F3F39F48881C6
:1002800087FD2E8180E880936C0006C08F818823D3
:1002900019F48E81821708F0822F8093610010C0BC
:1002A00080916C0087FF0CC0CE01B7D28F3F21F444
:1002B0008EE18093600004C0882311F010926100E9
:1002C00080918C00181614F410928C0080916000BC
:1002D00084FF58C0809161008F3F09F453C0182FEC
:1002E000893008F018E0811B8093610080917000D4
:1002F00098E8892780937000112391F180916C0018
:1003000087FF08C081E790E0612F16D2182F89304F
:1003100098F526C020918A0030918B0086FF0DC091
:10032000A1E7B0E080E090E0F901E80FF91FE49167
:10033000ED9301961817C1F708C0912FD901E1E795
:10034000F0E08D9181939150E1F71150812F90E071
:100350001F5F0196820F931F90938B0080938A00FA
:1003600081E790E0612F31D0612F6C5F6C3041F0FC
:100370008FEF8093610004C08FEF809361006EE186
:100380006093600094E186B3887131F49150D9F79D
:1003900010928D0010928700DF91CF911F910895E8
:1003A000A82FB92F80E090E041E050EA609530E05E
:1003B00009C02D9182279795879510F0842795275E
:1003C000305EC8F36F5FA8F30895EADF8D939D93C5
:1003D0000895A6E088279927AA9569F00197E1F387
:1003E000B399FCCFB39BFECF81E09927A6B30196CA
:1003F00011F0A871D9F70895CF93CFB7CF93C395D4
:10040000B39BE9F7B39B0BC0B39B09C0B39B07C079
:10041000B39B05C0B39B03C0B39B01C0D8C00F9270
:10042000DF93C0918900DD27C057DF4F012EB39BBA
:1004300003C0DF910F90E6CF2F930F931F934F933D
:100440002FEF4F6F06B303FB20F95F933F9350E00C
:100450003BE065C016B30126502953FDC89556B33D
:10046000012703FB25F92F7306B3B1F0502710279E
:1004700013FB26F906B22230F0F000C016B30127B4
:1004800003FB27F90126502906B22430E8F54F77FF
:10049000206816B30000F6CF50274F7D206206B2C9
:1004A000102F000000C006B300265029102713FBB0
:1004B00026F906B2E2CF4F7B06B3206400C0DACF44
:1004C00001265029187106B269F14E7F2160012F73
:1004D00016B328C0002650294D7F06B22260102F87
:1004E00029C0012650294B7F06B22460012F2DC060
:1004F00016B301265029477F2860000006B22EC09F
:100500004F7E06B3206130C0422706B349930026D0
:100510005029102706B24FEF13FB20F9297F16B39D
:1005200079F2187159F10126502906B2012703FB0F
:1005300021F9237F06B371F2002650293150D0F003
:1005400006B2102713FB22F9277E16B351F20126BB
:100550005029012703FB06B223F92F7C49F2000042
:1005600006B3102713FB24F90026502906B22F7971
:1005700039F270CF10E21ABF00271CC03B503195F2
:10058000C31BD04010E21ABF0881033C21F10B3499
:1005900011F1209187001981110F1213EDCF4A81BB
:1005A000441F093669F10D3211F0013E29F74F70F1
:1005B00009F0042F00938E003F915F914F911F919E
:1005C0000F912F91DF910F90CAB7C5FD18CFCF9132
:1005D000CFBFCF91189520918E00222369F31091FF
:1005E0008C001123D1F53430D2F130938C0020935C
:1005F0008800109189003BE0311B309389002FC0A7
:1006000000918C0001304CF50AE54F7049F43091AF
:10061000600034FD25C000936000C0E7D0E024C036
:10062000433049F030917B0034FD1AC000937B00C9
:10063000CCE7D0E019C03091A60034FD11C0009382
:10064000A600C7EAD0E010C0052710E000C021C016
:10065000052710E0C89508BB14C03AE501C032ED8B
:10066000032EC0E0D0E032E017B31861C39A08B39C
:1006700017BB58E120E84FEF20FF052708BB27955F
:1006800017951C3F28F700004552B0F720FF0527BB
:10069000279508BB17951C3FB8F629913A9561F745
:1006A000077E10918D00110F08BBC250D04011F091
:1006B0001093870010E21ABF086017B3177E402F0F
:1006C000477E54E05A95F1F708BB17BB48BB74CF7F
:1006D000FC018381813049F484E590E090938B00A4
:1006E00080938A0080915400089586E690E090936C
:1006F0008B0080938A0083E40895FC012081822F7F
:1007000080768032B9F49181892F8052823010F442
:100710008FEF0895923239F480916D00882319F497
:1007200082E080936D0027FD05C081E08093B200D8
:1007300080E0089580E00895FC0180916E00808340
:1007400080916F008183128213821482158288E067
:10075000868387E00895DC010BC0E92FF0E0E454C4
:10076000FF4F8D9180839F5F9F7790933D016150F4
:1007700090913D01662389F780913E018150891B4C
:100780008F77823018F48FEF80938C0008952EE0DD
:1007900088E190E00FB6F894A89581BD0FBE21BD09
:1007A00080E090E07AD18F3F09F081BF87EE88BB6F
:1007B00088E187BBA89584EC99E02CE931E0F90148
:1007C0003197F1F70197D9F717BA80EC92E190933E
:1007D0006F0080936E0080D084DC10926D001092C8
:1007E000B2007894A895B7DCC2D090916D0099239F
:1007F000C9F38091A60084FFF5CF923021F482E600
:1008000090E068E003C08AE690E062E09CDC8091C2
:100810006D00815080936D00E5CFFC018081809355
:100820006E00818180936F0080916E0090916F00C7
:1008300053D081E00895B299189501BB05B50FBD5D
:1008400009E00DBD07E000BF00E20BBF01B3189542
:1008500001BB0FB702BB0DB50A950DBD79F00BB505
:100860000695B29900680BBD13BB0FB51EB5011BF1
:100870000FBD13B302B30FBF01B3189500BF04BD82
:100880000BB50DBB00E40ABF00E60BBF02B30FBF00
:1008900001B3189501BBF09907C00BE40EB90EBB6C
:1008A00008B50FB901B3189500E40EB900E003BF15
:1008B00001B31895881F9795881F9795881F97955E
:1008C000881F9795881F9795881F9795881F9795DC
:1008D000881F9795892F08959C0181E080BD80E84D
:1008E00088B9B99ABA988BB78F7B8BBF1ABC13BEE5
:1008F00010BE80EE8EB984E58DB98FEF8FB9B90146
:100900007695679580E090E06C5E70418C4F9F4FCC
:1009100040E050E085D021502EBD8EB589BD1DBC74
:100920008EB590E0019695958795959587958195DB
:1009300085BD95B58EB5891718F08EB58F5F85BDCD
:1009400082E08ABD81E084BD90E499BF85B78C7F49
:10095000826085BF9ABF8BB780648BBF10923E01C7
:100960001092BB0010923C0110923D01089584B595
:10097000882379F49091BB00983058F48DB3E92F17
:10098000F0E0ED54FF4F80839F5F9093BB0081E0C8
:1009900084BD80917B0084FF12C06091BB00662300
:1009A00021F48091B200882351F083EB90E0CFDBFB
:1009B0008091BB0088708093B2001092BB0083B717
:1009C000882369F5E0913E0180913D018E1739F150
:1009D000F0E0E454FF4F80816DDF20913E012F5FF6
:1009E0002F7720933E0112BE9BE49EB91EBA982F2A
:1009F0009295907F9F6098BD8695F8948FB983E01B
:100A000083BF789480918C0087FF09C080913D015D
:100A10008095820F8F77823010F010928C000895AD
:100A200097FB092E05260ED057FD04D014D00AD00E
:100A3000001C38F450954095309521953F4F4F4F0D
:100A40005F4F0895F6F790958095709561957F4F6B
:100A50008F4F9F4F0895A1E21A2EAA1BBB1BFD01C9
:100A60000DC0AA1FBB1FEE1FFF1FA217B307E4078D
:100A7000F50720F0A21BB30BE40BF50B661F771FE5
:100A8000881F991F1A9469F76095709580959095C5
:100A90009B01AC01BD01CF010895E199FECF9FBB41
:0E0AA0008EBBE09A99278DB30895F894FFCF8E
:0C0AAE005AFFA12000000000020003001D
:00000001FF
